S02B0000433A2F576F726B2F736F6674776172652F4F70656E424C542F5461726765742F44656D6F2F41524DEF
S315080040008C010020FB41000865450008654500084D
S3150800401065450008654500086545000865450008CA
S3150800402065450008654500086545000865450008BA
S3150800403065450008654500086545000849450008C6
S31508004040654500086545000865450008654500089A
S31508004050654500086545000865450008654500088A
S31508004060654500086545000865450008654500087A
S31508004070654500086545000865450008654500086A
S31508004080654500086545000865450008654500085A
S31508004090654500086545000865450008654500084A
S315080040A0654500086545000865450008654500083A
S315080040B0654500086545000865450008654500082A
S315080040C0654500086545000865450008654500081A
S315080040D0654500086545000865450008654500080A
S315080040E065450008654500086545000865450008FA
S315080040F065450008654500086545000865450008EA
S3150800410065450008654500086545000865450008D9
S3150800411065450008654500086545000865450008C9
S3150800412065450008654500086545000865450008B9
S3150800413065450008654500086545000865450008A9
S315080041406545000865450008654500086545000899
S30908004150EE11AA555F
S315080041542B49072291438D462A482B492B4A00F0BE
S3150800416439F82B482B492C4A00F034F82B482C49AB
S315080041742C4A00F02FF82C482C492D4A00F02AF82E
S315080041842C482D492D4A00F025F82D482D492E4A4C
S3150800419400F020F82D482E49002200F026F82D4874
S315080041A42D49091A082903DB00220260043001603C
S315080041B41E481F49884205D00268043003B4904754
S315080041C403BCF7E700208646EC4600200021234A74
S315080041D49047FEE7884207D0521A05D00378013083
S315080041E40B700131013AF9D17047884202D0027046
S315080041F40130FAE770471A481A490160A8E700002F
S315080042048C01002058470008000000200000002008
S315080042146C4200086C4200085847000858470008D2
S3150800422400000020000000205847000858470008EE
S3150800423458470008584700085847000858470008D0
S315080042445847000858470008584700080000002047
S315080042540C0000200C0000208C00002001430008FC
S30D0800426408ED00E00040000827
S3150800426C80B582B000AF0121102000F051FA4FF44E
S3150800427C8053BB800323BB711023FB713B1D19466E
S3150800428C034800F06DF900BF0837BD4680BD00BF76
S3150800429C0010014080B582B000AF00F045F9786097
S315080042AC114B1B687A68D31AB3F5FA7F18D30F4BE0
S315080042BC1B78002B08D10D4B01221A704FF4805134
S315080042CC0B4800F017FA07E0084B00221A704FF457
S315080042DC8051074800F000FA034A7B68136000E037
S315080042EC00BF0837BD4680BD000000200400002032
S315080042FC0010014080B500AF00F004F8FFF7CAFFC4
S3150800430CFCE700BF80B584B000AF0023BB60002378
S3150800431C7B604F4A4E4B1B6843F0010313604C49B4
S3150800432C4B4B5A684B4B13404B60494A484B1B68DE
S3150800433C23F0847323F480331360454A444B1B687B
S3150800434C23F480231360424A414B5B6823F4FE0333
S3150800435C53603F4B4FF41F029A603D4A3C4B1B6817
S3150800436C43F4803313603A4B1B6803F400337B60C9
S3150800437CBB680133BB607B68002B04D1BB6840F279
S3150800438CDC529342EFD1324B1B6803F40033002BFB
S3150800439C00D1FEE7304A304B1B6843F0100313601C
S315080043AC2D4A2D4B1B6823F0030313602A4A2A4B0C
S315080043BC1B6843F002031360254A254B5B68536060
S315080043CC234A234B5B6843F400535360204A204B23
S315080043DC5B6843F4806353601D4A1D4B5B6823F48A
S315080043EC7C1353600923FB60FB68023B9B04FB6050
S315080043FC1749174B5A68FB68134343F480334B60D1
S3150800440C134A134B1B6843F08073136000BF104BA1
S3150800441C1B6803F00073002BF9D00D4A0C4B5B6834
S3150800442C23F0030353600A4A094B5B6843F0020303
S3150800443C536000BF064B5B6803F00C03082BF9D1DD
S3150800444CFFF70EFF00F056F800BF1037BD4680BDCB
S3150800445C001002400000FFF80020024080B483B030
S3150800446C00AF03463960FB7197F90730002B0BDA5E
S3150800447C0D49FB7903F00F03043B3A68D2B21201DB
S3150800448CD2B20B441A7609E0084997F907303A680C
S3150800449CD2B21201D2B20B4483F8002300BF0C37F8
S315080044ACBD4680BC704700BF00ED00E000E100E0AF
S315080044BC80B582B000AF78607B68B3F1807F01D39A
S315080044CC012311E00A4A7B6823F07F43013B5360C2
S315080044DC0F214FF0FF30FFF7C1FF054B00229A6002
S315080044EC034B07221A60002318460837BD4680BDC1
S315080044FC10E000E080B500AF0348FFF7D9FF0020B5
S3150800450C00F004F800BF80BD4019010080B483B0E8
S3150800451C00AF7860034A7B68136000BF0C37BD4652
S3150800452C80BC70470800002080B400AF024B1B68A3
S3150800453C1846BD4680BC70470800002080B400AF02
S3150800454C044B1B680133034A136000BFBD4680BC8D
S3150800455C704700BF0800002080B400AFFEE700BF1C
S3150800456C80B489B000AF786039600023FB61002302
S3150800457C3B610023BB610023FB6000237B610023A6
S3150800458CBB603B68DB7803F00F03FB613B68DB78A9
S3150800459C03F01003002B05D03B689B781A46FB6981
S315080045AC1343FB613B681B88DBB2002B44D07B684A
S315080045BC1B687B610023BB6138E00122BB6902FAE8
S315080045CC03F3FB603B681B881A46FB6813403B6188
S315080045DC3A69FB689A4226D1BB699B00FB600F229D
S315080045ECFB6802FA03F3BB60BB68DB437A691340CA
S315080045FC7B61FA69FB6802FA03F37A6913437B61F8
S3150800460C3B68DB78282B05D10122BB699A407B686D
S3150800461C5A6108E03B68DB78482B04D10122BB6958
S3150800462C9A407B681A61BB690133BB61BB69072B6E
S3150800463CC3D97B687A691A603B681B88FF2B46D9F5
S3150800464C7B685B687B610023BB613AE0BB69083316
S3150800465C012202FA03F3FB603B681B881A46FB68C7
S3150800466C13403B613A69FB689A4227D1BB699B00A8
S3150800467CFB600F22FB6802FA03F3BB60BB68DB43E3
S3150800468C7A6913407B61FA69FB6802FA03F37A6963
S3150800469C13437B613B68DB78282B05D1BB69083350
S315080046AC01229A407B685A613B68DB78482B05D116
S315080046BCBB69083301229A407B681A61BB690133CE
S315080046CCBB61BB69072BC1D97B687A695A6000BF85
S315080046DC2437BD4680BC704780B483B000AF786081
S315080046EC0B467B807A887B681A6100BF0C37BD46FF
S315080046FC80BC704780B483B000AF78600B467B8073
S3150800470C7A887B685A6100BF0C37BD4680BC7047F7
S3150800471C80B483B000AF78600B46FB70FB78002B37
S3150800472C06D00949084B9A697B6813438B6106E0E6
S3150800473C0549054B9A697B68DB4313408B6100BFBF
S3110800474C0C37BD4680BC704700100240C8
S705080041FBB6
